:100000000C9462000C948A000C948A000C948A0070
:100010000C948A000C948A000C948A000C948A0038
:100020000C948A000C948A000C948A000C948A0028
:100030000C948A000C948A000C948A000C948A0018
:100040000C9414020C948A000C948A000C948A007C
:100050000C948A000C948A000C948A000C948A00F8
:100060000C948A000C948A000000000024002700F1
:100070002A0000000000250028002B0000000000DE
:1000800023002600290004040404040404040202DA
:100090000202020203030303030301020408102007
:1000A0004080010204081020010204081020000012
:1000B0000008000201000003040700000000000027
:1000C00000001E0411241FBECFEFD8E0DEBFCDBF5D
:1000D00011E0A0E0B1E0E0EEFAE002C005900D9280
:1000E000A631B107D9F721E0A6E1B1E001C01D9228
:1000F000A93BB207E1F710E0C2E6D0E004C02197C7
:10010000FE010E946805C136D107C9F70E945E0250
:100110000C946E050C940000833081F028F481303B
:1001200099F08230A9F008958730A9F08830C9F09D
:100130008430B1F4809180008F7D03C08091800075
:100140008F7780938000089584B58F7784BD08955C
:1001500084B58F7DFBCF8091B0008F778093B00006
:1001600008958091B0008F7DF9CFCF93DF93282F32
:1001700030E0F901E255FF4F8491F901E656FF4F57
:10018000D491F901EA57FF4FC491CC23A1F081111A
:100190000E948C00EC2FF0E0EE0FFF1FE458FF4FA1
:1001A000A591B491EC91ED2381E090E009F480E019
:1001B000DF91CF91089580E090E0FACF1F93CF9325
:1001C000DF93282F30E0F901E255FF4F8491F901C8
:1001D000E656FF4FD491F901EA57FF4FC491CC2363
:1001E000A9F0162F81110E948C00EC2FF0E0EE0F89
:1001F000FF1FEE58FF4FA591B4918FB7F894EC9183
:10020000111108C0D095DE23DC938FBFDF91CF9111
:100210001F910895DE2BF8CFCF93DF9390E0FC0180
:10022000E656FF4F24918A579F4FFC018491882303
:10023000D1F090E0880F991FFC01E859FF4FA5917C
:10024000B491FC01EE58FF4FC591D491623071F426
:100250009FB7F8943C91822F809583238C93E881FB
:100260002E2B28839FBFDF91CF9108958FB7F894ED
:10027000EC912E2B2C938FBFF6CF1F93CF93DF9350
:10028000182FEB0161E00E940C01209739F460E027
:10029000812FDF91CF911F910C94DE00CF3FD105CC
:1002A00011F461E0F5CFE12FF0E0E255FF4FE4916A
:1002B000E33031F140F4E130B1F0E230E1F0C03848
:1002C000D1057CF7E4CFE73029F1E83059F1E4308B
:1002D000B1F780918000806280938000D0938B0082
:1002E000C0938A0004C084B5806884BDC7BDDF9117
:1002F000CF911F91089584B5806284BDC8BDF7CFAA
:1003000080918000806880938000D0938900C093A2
:100310008800EDCF8091B00080688093B000C093DA
:10032000B300E5CF8091B00080628093B000C093AD
:10033000B400DDCF8E50806480937C0080917A0081
:10034000806480937A0080917A0086FDFCCF809152
:1003500078009091790008958EE00E949A01E0E083
:1003600087369105A4F0E1E0853321E092077CF027
:10037000E2E0833022E0920754F0E3E0813D22E0A6
:1003800092072CF0E5E08F3993400CF4E4E0F0E0C4
:10039000EE0FFF1FE75FFE4F208131818091020148
:1003A000909103018217930779F08091AA019091AF
:1003B000AB01B9010E944D059093AB018093AA0156
:1003C00030930301209302010895CF92DF92EF92C0
:1003D000FF920F931F93CF93DF93CAE6D1E00AE217
:1003E00011E0C12CD12C7601D3940E947E04A70188
:1003F00096010E94D604699379930E947E04A70116
:1004000096010E94D604F801619371938F01F1E087
:10041000CA3ADF0751F7DF91CF911F910F91FF90FB
:10042000EF90DF90CF9008951F920F920FB60F922A
:1004300011242F933F938F939F93AF93BF938091FA
:10044000B5019091B601A091B701B091B80130917A
:10045000B40123E0230F2D3758F50196A11DB11DDE
:100460002093B4018093B5019093B601A093B70196
:10047000B093B8018091B0019091B101A091B20107
:10048000B091B3010196A11DB11D8093B00190936D
:10049000B101A093B201B093B301BF91AF919F910D
:1004A0008F913F912F910F900FBE0F901F90189535
:1004B00026E8230F0296A11DB11DD2CF789484B5F2
:1004C000826084BD84B5816084BD85B5826085BD50
:1004D00085B5816085BD80916E00816080936E00DE
:1004E00010928100809181008260809381008091D0
:1004F0008100816080938100809180008160809381
:1005000080008091B10084608093B1008091B00040
:1005100081608093B00080917A00846080937A003B
:1005200080917A00826080937A0080917A00816065
:1005300080937A0080917A00806880937A0010928C
:10054000C10062E084E00E940C0161E083E00E944F
:100550000C0161E08BE00E940C0162E081E10E94ED
:100560000C0161E08AE00E940C0162E089E00E94D7
:100570000C0183E28093B00081E08093B10082E8B7
:100580008093800089E1809381008FEF90E09093C9
:1005900087008093860060E08BE00E94DE008EE0A2
:1005A0000E949A01BC01990F880B990B6115710586
:1005B0008105910511F00E94CD040E94E5010E9481
:1005C000AC0144244A94512C88248A9423E0922E2E
:1005D000A12CB12C30E0232E30E0332E8FB7F894CD
:1005E000C090B501D090B601E090B701F090B8018D
:1005F0008FBFC092AC01D092AD01E092AE01F092FB
:10060000AF0181E10E94B500EC01019709F05FC0E4
:100610008091040181115BC00E94AC018091AA010C
:100620009091AB01019660910201709103010E94CB
:100630004D053C019093AB018093AA018FE00E948D
:100640009A012FEF30E0DC010E946105A5019401C1
:100650000E94D604660C771CF301E659FE4F6081B8
:100660007181629FC001639F900D729F900D112454
:10067000B2010E9439058B018AE00E943D01B80158
:1006800083E00E943D0180E10E949A012FEF30E05B
:10069000DC010E946105A50194010E94D604F301CA
:1006A000E65DFE4F80819181821793070CF0A4C014
:1006B0002AE0C20ED11CE11CF11CC0922601D0928E
:1006C0002701E0922801F09229011092010181E0B6
:1006D000CD2B09F480E08093040189E00E94B500ED
:1006E000EC01019731F480910001811102C00E9458
:1006F000E50181E0CD2B09F480E080930001809139
:100700000101C090AC01D090AD01E090AE01F0903D
:10071000AF01811175C08091260190912701A091B0
:100720002801B0912901A7019601281B390B4A0B1A
:100730005B0BDA01C901B7FD0FC061E08BE00E94DD
:10074000DE00C0922201D0922301E0922401F092B7
:10075000250131E03093010184E00E94B500109240
:1007600020011092210190911F01891751F080936F
:100770001F01C0921A01D0921B01E0921C01F0925D
:100780001D0180911A0190911B01A0911C01B09153
:100790001D01C81AD90AEA0AFB0A80911601909134
:1007A0001701A0911801B09119018C159D05AE0596
:1007B000BF05B0F490911E0180911F01981781F040
:1007C00080931E01911103C021E0813009F020E0E7
:1007D00020932001913009F4811190E09093210140
:1007E0008091210181110E94E5012114310409F455
:1007F000F5CE0E940000F2CE32E03093010167CFC7
:10080000813009F0A9CF8091220190912301A0911C
:100810002401B0912501A7019601281B390B4A0B31
:100820005B0BDA01C9010397A105B10508F494CF68
:1008300060E08BE00E94DE0032E08CCFE6E1F1E088
:1008400082E390E0A0E0B0E080839183A283B38351
:10085000148215821682178281E080878187128632
:10086000138608958F929F92AF92BF92CF92DF929C
:10087000EF92FF92CF93DF93EC01688179818A81B7
:100880009B81611571058105910521F464E279ED83
:100890008BE597E02DE133EF41E050E00E94D60474
:1008A00049015A019B01AC01A7EAB1E40E94F50499
:1008B0006B017C01ACEEB4EFA50194010E9403052D
:1008C000C60ED71EE81EF91EF7FE06C081E0C81A44
:1008D000D108E10880E8F80AC882D982EA82FB825E
:1008E000C701B6019F77DF91CF91FF90EF90DF9026
:1008F000CF90BF90AF909F908F9008958F929F92CE
:10090000AF92BF92CF92DF92EF92FF92609105017A
:1009100070910601809107019091080161157105A0
:100920008105910521F464E279ED8BE597E02DE1F5
:1009300033EF41E050E00E94D60449015A019B0187
:10094000AC01A7EAB1E40E94F5046B017C01ACEEB6
:10095000B4EFA50194010E940305C60ED71EE81E40
:10096000F91EF7FE06C081E0C81AD108E10880E848
:10097000F80AC0920501D0920601E0920701F092B8
:100980000801C701B6019F77FF90EF90DF90CF90ED
:10099000BF90AF909F908F900895609305017093E2
:1009A000060180930701909308010895052E97FB97
:1009B0001EF400940E94ED0457FD07D00E94080524
:1009C00007FC03D04EF40C94ED04509540953095FF
:1009D00021953F4F4F4F5F4F0895909580957095AB
:1009E00061957F4F8F4F9F4F08950E942A05A59FC5
:1009F000900DB49F900DA49F800D911D112408951A
:100A0000B7FF0C94F5040E94F504821B930B089524
:100A1000A1E21A2EAA1BBB1BFD010DC0AA1FBB1F02
:100A2000EE1FFF1FA217B307E407F50720F0A21B74
:100A3000B30BE40BF50B661F771F881F991F1A94E1
:100A400069F760957095809590959B01AC01BD010B
:100A5000CF010895A29FB001B39FC001A39F700D65
:100A6000811D1124911DB29F700D811D1124911DB6
:100A70000895AA1BBB1B51E107C0AA1FBB1FA617E5
:100A8000B70710F0A61BB70B881F991F5A95A9F737
:100A900080959095BC01CD01089597FB072E16F423
:100AA000009407D077FD09D00E94390507FC05D0D6
:100AB0003EF4909581959F4F0895709561957F4F75
:100AC00008950E942A05B7FF0895821B930B08958D
:100AD000EE0FFF1F0590F491E02D0994F894FFCFDD
:100AE00001020800010100000003000400050008E5
:060AF000001000200000D0
:00000001FF
